:100000000C9434000C943E000C943E000C943E0082
:100010000C943E000C943E000C943E000C943E0068
:100020000C943E000C943E000C943E000C943E0058
:100030000C943E000C943E000C943E000C943E0048
:100040000C943E000C943E000C943E000C943E0038
:100050000C943E000C943E000C943E000C943E0028
:100060000C943E000C943E0011241FBECFEFD4E050
:10007000DEBFCDBF0E9440000C9454000C940000E1
:10008000209A81E085B9E3EDF0E33197F1F700C004
:10009000000015B8FFE32DE033E0F1502040304080
:0C00A000E1F700C00000EECFF894FFCFA5
:00000001FF
